:0600000018308A00002FF9
:08000800FF00030E8312FE004D
:100010000A08FA008A018C1E26280408FC003C0805
:1000200084001A08243A031D17283F1522281A08AD
:1000300080000008BC0A3C1A3C120D3A2011031D36
:10004000242820154030BC007C0884007A088A00EF
:0A0050007E0E8300FF0E7F0E0900F4
:100080008A150A160A2F8A150A160B2F4928E22903
:100090003D2C210E07398207D02CD02C102B102B91
:1000A000452B452B942821080F3982076628AE2C52
:1000B000B12CBA2CB42CB72C452B872D972D972D0E
:1000C000B22DB82D9D2DBD2DC72DD82D22083F391D
:1000D0008207552B4B2BDF29572BE529592B5B2BFF
:1000E000172BE52C3F2DE12B5D2BCE2CDC2C402C4F
:1000F000772C8B2C8B2C8B2C8B2C9B2C9A2C852C43
:100100007F2C882C822CD62CD92C932D8C2DE02C56
:10011000702CD429DD2D82070134023404340834D4
:100120001034203440348034210803398207932C62
:100130008E2C452B22080F398207E62DE92DEC2D58
:10014000EF2D452B452B502BE12DF22DF72D452B77
:10015000452B452B452B452B452B6430BE00B22843
:100160000A30BE00C020BE0BB22808000530C128EE
:100170000230C1280030C1280330C1280430C12812
:10018000063083168100831281016400473001022A
:10019000031CC528003083168100831200341D2201
:1001A000AE001530AD002D08073A0319DF28CF3017
:1001B0002E020318DF280530AE07AD03D328063022
:1001C00095002D08831692008312B028950108002F
:1001D0007B13CF208316813087008312871107128B
:1001E00087102121B801B90187166921B020871233
:1001F0008714B0204F21871087166921B0208712FD
:1002000087141D22AD00B0202322AE0021218710CB
:1002100087166921B02087128714212900344621CE
:1002200028212821282128212821282128214F215F
:100230003F30A1057F30A2053A219921B801B901CB
:1002400008008101640027300102031C22290034C8
:10025000B90A0319B80A0630AF000630A5002F1CF2
:1002600007122F180716871531228711AF0CA50B1F
:100270002F29003421083F39B0002208B100BF10F7
:10028000211BBF140230A0190330211B00302C2188
:100290004A216F213008A1003108A2000034043047
:1002A000A01905302C218711071683160716831213
:1002B000A101A2011030A50087150310A10CA20C0A
:1002C000071AA1178711A50B5C290310A10CA20C1A
:1002D00021136400831607128312071200340310DF
:1002E000A20DA10D1030A500871522180716221C9B
:1002F0000712A10CA20C8711A50B74290034083039
:100300002C21B620BE20B820080018302C21BE2099
:10031000BC20BA20BA200800831612088312B50048
:10032000BE201130350203180800BE20B50A9129FD
:1003300008002013640021083F39B0002208B100F2
:100340000430A01905302C21212153214114FF3004
:100350002206031D4110A019B2293F30A105210634
:10036000031D41104A210230A01903302C214A21DB
:100370006F21411CBD298521BE297F210430A01990
:1003800005302C212121532131082206031DCE29BD
:10039000A0194F293008210603194F290E30A1005A
:1003A000EE30A20020170034E820AD20462128219D
:1003B000282128212821282128214F21402B4F2185
:1003C0002821452B3A21BF18452B99212821452B5F
:1003D000BD003D0EEC213D080F393038AF00393CEF
:1003E0000318F4290730AF072F08AF006430B700B7
:1003F0003F19FF29B60B022AB70B022A00000000A2
:10040000861608006400061AF8292F089900212191
:1004100083169818092A981C0B2A83128612B70192
:100420003F19FF29061E162A86160800BE0B102A41
:100430006400B70B102A86160800C130242AD13078
:10044000242AE130242AC9309F0031221F1531228D
:100450001F19282A21211F1531221F192D2A312267
:100460001E0864000800C0303A04F5003B08F6009E
:100470002012A501071E492A87156400071E492A74
:10048000A60B3D2AA50B3D2A2016831607168312BC
:100490000800E030F1008122812281228122A50121
:1004A000F70187118122A0108715071A5A2AA50B78
:1004B000552A442AA501A60B612A6400A50B612ACE
:1004C000442AF70A0319A014071A5B2A871181220C
:1004D00087159622F113F51BF1170310071A031461
:1004E000F60DF50D8316071283120712F11B07167E
:1004F00087119622831607168312F10A711E682A45
:10050000452A6400BF1B892AF10AF11D812AF111D5
:10051000080064000000000000000000000000006F
:100520000000F10A711F892A711308007708A600DC
:100530006400BF1B9F2AA60B992AA01C0800640018
:10054000000000000000000000000000A60B9F2A31
:10055000A01C08006400AC2AA60BAA2A0800730895
:10056000F6006230F500382281227008F600613012
:10057000F500382281227408F6006330F500382235
:100580008122F6006030F5003822812A28213808BF
:100590003A06031DC62A39083B06031DC62A080071
:1005A0004030F50032197514A7132713B218A71796
:1005B000321827172708F60008002208B200A70102
:1005C000A0308400D02238228122A70AD0223822EB
:1005D00076088000840A0408E03A031DE42A8413A4
:1005E0007F30F500F601382208004030201B4130F2
:1005F000F5003208F6000800831603178C13FB1A67
:100600008C170C140000FF3EFF3EFF3EFF3E6400CF
:0606100083120313080031
:1006200021081F39BA002208BB00C722452B0B172F
:10063000E820AD2046212821282128212821282111
:10064000282128214F210E30A105CF30A2053A21C3
:1006500099217F30A100FF30A2003A210730A70086
:1006600006302C21A70B302B01302C2107302C21F8
:1006700008302C218C2101302C2107302C21B02076
:100680007B13E6208710871621212108F5212208F7
:10069000F521411043287B13E6208710871621217E
:1006A0008316993087008312402BE820452B2821A0
:1006B000452BA011452BA015452B831680308700B4
:1006C0008312A201A101503084001D228000840AFF
:1006D0008712C0202322AF008000840A57302F02E7
:1006E0000318221413302F02031C22148716B02083
:1006F0002322AF008000840A0F302F020318A214B7
:10070000CF2087128714AD2023228000840AAF00F7
:10071000BB302F02031822158D302F02031C221527
:10072000871021218716BC20071000008618A2150B
:1007300007140000861CA215071007162122C020EE
:100740002122AF00B0008000840A77302F02031C02
:10075000221607122122C0202122AF008000840A25
:100760000F302F020318A21687151F22C0201F2248
:10077000B100AF008000840A7F302F02031C2217D3
:1007800087111F22C0201F22AF008000840A0D3075
:100790002F020318A2178316813087008312E620E8
:1007A0002208E5007B13FB17E22BE6208710871653
:1007B000212183169930870083126508A200A101C8
:1007C000452BFB13F0018316F0018312E8204F2123
:1007D0002108EA002208EB00E620B020E8202830BB
:1007E000A1000030A2003A219921C020E620B020CB
:1007F000871183160716871183120530B6008716F6
:10080000B0208712B020871521218711B020183021
:10081000F6006130F500382281228030F500F601C3
:100820003822201E152CB60BFF2BE8206A08A100E9
:100830006B08A2003A219921C020E620B02087153C
:10084000831607168312B02087108716B0208712F0
:10085000B0200730B6002121071E332CB60B2B2CFD
:10086000FB1BD52B392C7B17FB1BD52B452C871558
:100870008122000000008711452B3F14C020452C29
:10088000FF30F500F6013822812220107F30F5007C
:10089000F6013822201A392C75081F39A300760872
:1008A000A4008122F501F601382281221030F500E2
:1008B000F60138227608F20081222030F500F60198
:1008C00038227608F00081223030F500F601382217
:1008D0007608F3007F30F500F60138227608F40040
:1008E0002308A1002408A2003F1C452B4328201404
:1008F0003F103322C020A1010130A200452B720815
:10090000A200452B7308A200452B7008A200452BBE
:100910007408A200452B2208F800452B2208F60097
:100920006530F500A32C2208F6006430F50038226B
:100930008122452BF30A4030F5007308F600F818C1
:1009400075147818F617382281227F30F500F601E9
:1009500038220030F5217608F52143282208F200DC
:10096000452B2208F300452B2208F000452B2208D6
:10097000F400452B2208C1225030F5007308F60020
:10098000F81875147818F617382281227208C122D7
:100990007F30F500F60138228122452BAF22452B0E
:1009A00021081F39BA002208BB00452B8710871683
:1009B000452B87108712452B871521218711452B41
:1009C000A101A20120182214452BE8200730FB18B2
:1009D000EC2C1F307B180E30BA00E0307B1C00304E
:1009E000BB00C72203171730FB18F92C0F307B18F8
:1009F00006308F00E0307B1C00308D000313FB16A7
:100A00007B12FC2203170E080313A10003170C0826
:100A10000313A2008A013A219921282103178D0A84
:100A200003198F0A0F080313FB1C182D083A1B2DFE
:100A30007B18083A7B1C103A031D012DFB1246213E
:100A400028212821282128212F30FB182A2D2F305A
:100A50007B182E30A100E0307B1C0030A2003A2130
:100A600099212821282128214F213730A1053F3005
:100A7000A2053A2199210000402B0000452BE820D7
:100A8000A4010830FB18472D10307B1C2030A30038
:100A90004F21282121083F393F3A031D852D220A85
:100AA000031D852DA40B482DA30B482D7F30A100DD
:100AB000FF30A2003A210630A4004F21282121084E
:100AC0003F393F3A031D852D220A031D852DA40BB6
:100AD0005D2D28214F21282121083F393F3A031D50
:100AE000852D2208FF39FF3A031D852D0830A4000B
:100AF0004F21282121083F393F3A031D852D220A25
:100B0000031D852DA40B782D402BCE21402B2208D0
:100B1000831692008312C0202322A200831612089B
:100B20008312A100452B1D22A200A101452B2013F9
:100B3000211820172208B200452B2208A700A03058
:100B40008400F52238228122B20AF5223822760862
:100B50008000840AA70BA32D84137F30F500F601D3
:100B60003822B32DDD220030F5213208F52140284E
:100B7000BF1322080319BF17452B2208A700A03076
:100B800084000008F521840AA70BC12D4028220803
:100B9000A700A03084000008990083169818CE2D75
:100BA000981CD02D83122121840AA70BCB2D40281D
:100BB0000230A1003030A200452BA1010130A2007B
:100BC000452BA101A2017B1B2214452B7B10FB109E
:100BD000452B7B14FB10452B7B10FB14452B7B1402
:100BE000FB14452B6808E6006908E700452BAE01B9
:100BF000AD01FB1669086706031D072E6808660627
:100C0000031D072E2D08A1002E08A200452B680801
:100C100003178F000313690803178D000313FC22C9
:100C2000031003170C080313AE070318AD0A0317CC
:0E0C30000E080313AD07E90A0319E80AFA2DAE
:100DC000ED00030883160317F00083006D088312FB
:100DD0000313ED0083160317ED000408EE000A0864
:100DE000EF001F308A000E08EB0003178316E03077
:100DF000EC0506178613831286138316EC0A6C1D06
:100E0000FE2E6C1183126400061B032F6400061F64
:100E1000062F86178316EC0AEC1D0B2FEC1183129C
:100E200086136400061B112F6400061F142F031085
:100E30008316EC1B031483128613031C8617061BF0
:100E40001F2F831686176400EC0A83120310861B7B
:100E500003148316EC130318EC1783126400061FA7
:100E60002E2F86138316861303106B1B0314831215
:100E70008613031886176400061B3B2F83168617FC
:100E800003108F0DEB0DEC0A83120310861B031465
:100E9000831603180F146C1E2D2FEC1F602F6B0888
:100EA0008E006E0884006F088A0070088300831625
:100EB0000317ED0E6D0E701F0313F01E8312080052
:100EC0006B0E073982078A2F8E2F8C2F902F762F4B
:100ED000822F6B2F7D2F6B0807398207922F982F57
:100EE000952F9B2F9E2FAA2F7D2F7D2F83136B185D
:100EF00083170F08840000088F0083126400061F08
:100F00007E2FF52E83136B1883170F0884006D084E
:100F100080007D2F6D087C2F6E087C2F70087C2F41
:100F20006F087C2F0F08ED007D2F0F08EE007D2F3E
:100F30000F08F0007D2F0F08EF007D2F0F088312A0
:100F40008C0083168C130C1555308D00AA308D0043
:100F50008C147D2F0F0883128D0083168C130C14B4
:080F600083120C0883167C2F9C
:101E00007011031970157013031B7017F012831AE9
:101E1000F01603178316ED006430F00503089B39B4
:101E2000F0040408EE000A08EF001F308A000E08D4
:101E3000EB0003178316E030EC05061786138312B8
:101E400086138316EC0A6C1D222F6C11831264001A
:101E5000061B272F6400061F2A2F86178316EC0AFD
:101E6000EC1D2F2FEC11831286136400061B352FF7
:101E70006400061F382F03108316EC1B0314831213
:101E80008613031C8617061B432F831686176400D0
:101E9000EC0A83120310861B03148316EC13031839
:101EA000EC1783126400061F522F861383168613C5
:101EB00003106B1B03148312861303188617640028
:101EC000061B5F2F8316861703108F0DEB0DEC0A90
:101ED00083120310861B0314831603180F146C1E41
:101EE000512FEC1F842F6B088E006F088A006E083C
:101EF00084007008830083160317ED0E6D0E701FAB
:101F00000313F01E831208006B0E07398207AE2FF1
:101F1000B22FB02FB42F9A2FA62F8F2FA12F6B087F
:101F200007398207B62FBC2FB92FBF2FC22FCE2F54
:101F3000A12FA12F83136B1883170F0884000008AB
:101F40008F0083126400061FA22F192F83136B18B2
:101F500083170F0884006D088000A12F6D08A02F43
:101F60006E08A02F7008A02F6F08A02F0F08ED009B
:101F7000A12F0F08EE00A12F0F08F000A12F0F08CE
:101F8000EF00A12F0F0883128C0083168C130C1501
:101F900055308D00AA308D008C14A12F0F088312AC
:101FA0008D0083168C130C1483120C088316A02F3B
:102E00007011031970157013031B7017F012831AD9
:102E1000F01603178316BD006430F00503089B39D4
:102E2000F0040408BE000A08BF001F308A000E0824
:102E3000BB0003178316E030BC0506178613831208
:102E400086138316BC0A3C1D222F3C11831264009A
:102E5000061B272F6400061F2A2F86178316BC0A1D
:102E6000BC1D2F2FBC11831286136400061B352F47
:102E70006400061F382F03108316BC1B0314831233
:102E80008613031C8617061B432F831686176400C0
:102E9000BC0A83120310861B03148316BC13031889
:102EA000BC1783126400061F522F861383168613E5
:102EB00003103B1B03148312861303188617640048
:102EC000061B5F2F8316861703108F0DBB0DBC0AE0
:102ED00083120310861B0314831603180F143C1E61
:102EE000512FBC1F842F3B088E003F088A003E08EC
:102EF00084007008830083160317BD0E3D0E701FFB
:102F00000313F01E831208003B0E07398207AE2F11
:102F1000B22FB02FB42F9A2FA62F8F2FA12F3B089F
:102F200007398207B62FBC2FB92FBF2FC22FCE2F44
:102F3000A12FA12F83133B1883170F0884000008CB
:102F40008F0083126400061FA22F192F83133B18D2
:102F500083170F0884003D088000A12F3D08A02F93
:102F60003E08A02F7008A02F3F08A02F0F08BD001B
:102F7000A12F0F08BE00A12F0F08F000A12F0F08EE
:102F8000BF00A12F0F0883128C0083168C130C1521
:102F900055308D00AA308D008C14A12F0F0883129C
:102FA0008D0083168C130C1483120C088316A02F2B
:063BFA0002003000010092
:103C00008101640027300102031C012E0034831659
:103C100006118312A70164008C1A1E2EBE0B0B2EF8
:103C2000A70B0B2E831606158312A70164008C1AAE
:103C30001E2EBE0B162EA70B162E072E8A110A1249
:103C4000BE208A150A168C121A08553A03193C2E02
:103C5000A01E382EA012831619080B3A0B30031938
:103C600003309900831218121816033A031D072E09
:103C7000A01618121816072E75304B268316061537
:103C800083124030BC00C0308B00352F21084B26FA
:103C900022084B26352FAF006430B7003F19552E50
:103CA000B60B582EB70B582E0000000086160800E1
:103CB0006400061A4E2E2F089900000083169818EB
:103CC0005F2E981C612E83128612B7013F19552E64
:103CD000061E6C2E86160800BE0B662E6400B70BFF
:103CE000662E86160800BF112F300002031CBF1578
:0E3CF0003A300002031C080007308002080072
:103E00000C2F8A110A1246288A110A1247288A1191
:103E10000A124828352F392FC03087002F308500EF
:103E2000FB30860095010F3097008316DF30860047
:103E3000993087003F30850003309F0020308C0090
:103E400024309800033099008101153092008312CC
:103E500012158710871690309800A001BF01FB0152
:103E6000F801BA01BB01A012072EC0308B00403010
:103E7000BC0064003F193F1118191A08981C422F02
:103E800018121816201C462F071E072F201D392F29
:103E900020113F104030840000080319840A732663
:103EA000BF19392F000EF039A100840A7326BF19FB
:103EB000392F00080F39A104840A7326BF19392F3E
:103EC000000EF039A200840A7326BF19392F0008AA
:103ED0000F39A2042108E039403A0319E62F7B1D6F
:103EE000752F2108C0390319F02F7B112108633A7F
:103EF000031D842F2208563A0319892F2208653A98
:103F0000031D842F7B15462EFB117B11A11B042F53
:103F1000012FFB15462E83160F308100831264009B
:103F2000690803178D000313680803178F00031334
:103F3000220803178C000313210803178E00831631
:103F400003178C170C158B1355308D00AA308D007C
:103F50008C140000FF3EFF3EFF3EFF3EFF3EFF3E53
:103F6000FF3EFF3EFF3EFF3EFF3EFF3EFF3EFF3E69
:103F7000FF3EFF3EFF3EFF3E0C118C1383016400A9
:103F80000D1EBF2F0D1283168101831269080317BE
:103F90008D000313680803178F00DC2783120317B3
:103FA0000C080313A20003170E080313A100080056
:103FB000E90A0319E80A0800831603178C170C1482
:103FC0000000FF3EFF3E8C138301080021081F39CB
:103FD000E8001F3A031968122208E900C627462E96
:103FE00068081E391E3A0319FC2F6808031DFB2FB1
:0C3FF0006908C039031D8B27D827462E16
:02400E002D2F54
:00000001FF
